:100000000128831600308100E830850088308600A2
:10001000831212308500403086009B01103094001E
:10002000303084008001840A940B12281030940030
:1000300040308400AE012E088900FA238000840A33
:10004000AE0A940B1B280512AF019901A6018C0181
:100050008D01A9011D300B118207AE28D428C028BC
:10006000CB28D728DE2801280128012803291E29AA
:10007000212938295A299029B0295F298B2B6B2AED
:10008000682AE42A832AE129ED29942BE82BEF2B17
:10009000FC290C2A63286928402A4E2AA02BAA2B67
:1000A000132B4D2B820700340134053400340934FE
:1000B0000034003400340D340B1D5C28A800C93016
:1000C000810028082B2805160130CB3081001E3016
:1000D0005C280516143094008320143094008C2082
:1000E0009908031975288616762886121B0A07397F
:1000F0009B00012123213A219421B2211B080339BD
:100100000319C32370289001910103309600FE204B
:100110009120940B832808000A306322940B8C28CA
:100120000800013065221030840016088F008F030C
:100130008F030008840A0006840A8F0B9B28800026
:10014000103084000B1DA228D93081000B119C0AAD
:10015000A91FE2200930970000305C2805120B1D12
:10016000AF28D93081000B11A91BE220970BB928C9
:10017000D928800D031CBE2801305C2802305C2881
:1001800005160B1DC128D93081000B119C0AA91F2F
:10019000E22003305C2805120B1DCC28D9308100E9
:1001A0000B11A91BE220B628051604305C280512A5
:1001B000B628840A0930970005305C280516960B8E
:1001C000A22808001C1B9C0129087F391C02031867
:1001D000F8281C08AA00AA0C2A0C0F39303E890006
:1001E000FA23AA00F920AA0BF228F53081000B119E
:1001F00008001C308F008F0BFB2808000A30652296
:10020000080009305C2805129D011B181D179B185A
:100210001D161B199D161D088E389D00851008306F
:10022000A3009D0D031C162905151729051105149A
:100230000510A30B112985140A305C2805160B3014
:100240005C28051208009E010730970085100514F0
:10025000051005140510851D2F29031430290310DE
:100260009E0D05140510970B2B2985140C305C2866
:1002700005160800AE01F83086051B08860402301A
:10028000960002309400043098000616000000002A
:100290000000861D4D2903144E290310061200008C
:1002A0000000AE0D980B4529940B582910305C289E
:1002B0000D305C28051243292E089F0041290516A0
:1002C000960B5C292E08A0009F1F67299229A00980
:1002D0002008AE00AE0E0F30A005AE050A30AE0805
:1002E00003197529A007AE036F299B08031D7B29FD
:1002F0000314AF0D7D290310AF0D061600008619FB
:1003000086292F080D05031926168D292F080D059E
:1003100003198D292F0999058D0506120E305C28C9
:1003200005120800A00175291F09A100261AAE298F
:100330002F080D05031DAE2938301B07840020301F
:1003400080070F302105031DA7290016AE29001ACA
:10035000AA29AE290F302105800600120F305C2833
:100360000516080030301B0784009F1FBE292F0987
:100370009905801F622A80130008FF2AA017200811
:100380000002031DC729261EC629032B6F2A9E08BB
:100390000319D3292F099905801F622A2F0999056E
:1003A0000008A0006F2AAB013030840002309400B6
:1003B000200800020319AB0A840A940BD8291630CE
:1003C0005C28051204309400200800020319AB0ACF
:1003D000840A940BE42917305C2805160230940037
:1003E000200800020319AB0A840A940BF029AB0819
:1003F000031D3E2A1B305C280512303084001B0888
:100400008407801F082A00087F39031D082AA901D4
:100410002F0999051C305C28051619222008AE000A
:100420000008A0002E088000A01F622A9E012C2236
:100430006F2AA0135A302002031926145B302002C1
:100440000319A6145C302002031926155D30200222
:100450000319A615A0170800A0135A30200203198B
:1004600026105B3020020319A6105C30200203190D
:1004700026115D3020020319A61108001F305C28E8
:100480000516303084001B08840700087F39031DDF
:100490004A2AA9012F08990420305C280512801BE4
:1004A000532A0530632A80130008A0002C229E01E5
:1004B0009E0A6F2AFF3090000030910003309600B2
:1004C0009120E62A053065225A2A950013305C28CF
:1004D000051212305C280516950B662A0800A01339
:1004E000A008031D7D2A1E08A900A90C1F1E7A2A38
:1004F000A9177B2AA9130330622A5B2BA0080319D2
:100500007B2A15305C28051260301F05AE000319E8
:10051000902A60302E020319902AAE1E9F2AD12AFB
:100520002008900090133F3091001E0892001F1A7F
:100530009B2A92179C2A921304309600E22A2008E4
:100540009000901391011E030319CE2A03301E055B
:10055000AA001E089D009D0C9D0C1F309D050230B9
:100560001D02031CCC2A38301B078400000E8F00AC
:100570000F0C03392A02031CC62A0319C62A861F38
:10058000C62A1F309D051D02031D9D0A1D0C031860
:1005900011169104F222E22A9D01C62A1E0891003A
:1005A000CA2A2008900090131E030319ED2A9E0CFE
:1005B0009E0C1E0C9100111238301B07840000188D
:1005C0001116F22214305C2805169120261F08000F
:1005D000A61FF02A05306522782B1E089100E12A1B
:1005E000261308001F1AF62A9116F72A9112911362
:1005F00011170330960008001F1EF62AF42AA000E7
:100600009E019E0A2C2221080F398F000319542BBA
:1006100009300F020318542B0F0852200319542BD2
:100620008F0023305C2805128F03AE019A019801D8
:1006300020088E008E13980A0F08403E84000008A0
:100640000319322B7F390E020319292B8E08031D43
:100650002B2B18089A00980A840A05301802031DEB
:100660001F2B352B1808AE002B2B043084021A08E0
:1006700003193D2B1A038407582B2E080319542BFA
:100680002E0384070E0880001F1A801700088800B8
:1006900040300402890024305C20051683160815BA
:1006A000F1232F088D0499042612043065226F2A45
:1006B00080018801482B5A302002031C862B033C02
:1006C000031C862BA61726171F08A7005A30A00266
:1006D0000310A00DA00D403020079A0004309800B0
:1006E0001A0884000008031D7A2B980B782B842BA2
:1006F0009A0A702BA0002708A01F7F2B103A9F009A
:10070000A013043065227E2AA6137A2BAB01403059
:10071000840011305C280512B723003C0319922B8A
:100720002618AB0A18305C28051602306522840AA8
:10073000B723003C03199E2BA618AB0A21305C2876
:100740000512840AB723003C0319A82B2619AB0A0B
:1007500022305C280516840AB723003C0319B22B0B
:10076000A619AB0AAB0803197E2A0430632A0430A9
:10077000A30000087F39200203190134A30BC12B09
:100780000034840AB92B0C0A07398C008C08031D2D
:10079000CC2B013094008C2030300C078400801F5B
:1007A000E62B00089000901390080319E62B3830D0
:1007B0000C07840000080F399100910C03181116E2
:1007C000911703309600FE209120080019305C2814
:1007D000051208308407E03080051A305C280516C1
:1007E000080055308900AA308900881400000811DB
:0E07F0008312080083160814831208080800FC
:02400E00F23F7F
:1042000000000000000000000000000000000000AE
:10421000000000000000000000000000000000009E
:104260000700080009000A000C000E0010001300EF
:1042700018001D002500300041005D009100FF0086
:00000001FF
